:10000000830100308A007928FC0003088301C000C6
:100010007008BE007108BF0083018B1C4628861C37
:100020001328013014280030F0008316011F1A280D
:1000300001301B280030F006031D2428FF308312F6
:10004000AA07031CAB0328288312AA0A0319AB0AC8
:10005000831640308106011F43288312861C3428F2
:100060000E08AC000F0840280F08F1000E08F00041
:10007000F009F109F00A0319F10A7008AC007108DF
:10008000AD008E018F018B10831203130C1C4D28C1
:10009000FF30AC007F30AD000C108C1C7028A1012B
:1000A000A10A2608A8002708A9002408A6002508F8
:1000B000A7002208A4002308A5002A08A2002B08F4
:1000C000A300A00803196628A00368286430A000D4
:1000D0000A30200203186E2807146F2807108C10AE
:1000E0003E08F0003F08F10040088300FC0E7C0E43
:1000F0000900203084003E3082208301482D040610
:0C0100008001840A0406031D7F280034DF
:1006A200813083019F00FF308316850080309F00D8
:1006B2008312080020308301940083168712871169
:1006C20087100711831208008301B0000F30B005B4
:1006D2000A30300230080318702B303E0800373ED3
:1006E200080083160313981C722B0D308312990095
:1006F2008316981C792B0A30831299000800C030A7
:1007020083160313870422309800903083129800D6
:1007120083160C128C1618150A30990018128312BF
:100722000800F401F5010310F30CF20C031CA02BDA
:100732007008F40771080318710AF5070310F00D29
:10074200F10D7208730403190034942BF430830101
:10075200B0000130B100FF30B007031CB103310813
:100762003004FF30031DAD2BB007031CB103310869
:10077200300403190800A72B83013908F3003A0853
:10078200F4003B08F500F0012030F1004130F200A6
:10079200D126CD30F3004C30F4004230F50038273A
:1007A20079277008BC007108BD00803AF0008430DF
:1007B2007002003003193C02031CE32BFF30BC0023
:1007C2000330BD00BD1FE72BBC01BD0107118C1119
:1007D2003D08F1003C08F0000530F200710DF10C0B
:1007E200F00CF20BEF2B700893008C1DF62B8C1182
:0E07F2003C08F0000310F00D0310F00D031092
:10080000700D93008C1D022C071508008301390818
:10081000F3003A08F4003B08F500F0012030F10045
:100820004130F200D126CD30F3004C30F40042309C
:10083000F500382779277008BC007108BD00803AA0
:10084000F00084307002003003193C02031C2C2C91
:10085000FF30BC000330BD00BD1F302CBC01BD010A
:1008600087108C113D08F1003C08F0000530F200C3
:10087000710DF10CF00CF20B382C700893008C1DEC
:100880003F2C8C113C08F0000310F00D0310F00D0C
:100890000310700D93008C1D4B2C871408008301EE
:1008A0003008B0003108B100B11F622C8316981CCB
:1008B000562C2D3083129900B009B109B00A0319E2
:1008C000B10A682C8316981C622C2B308312990075
:1008D0003008B0003108B1003230B200D4258316A0
:1008E000981C6F2C83123608652399008316981C78
:1008F000762C83123508652399008316981C7D2C6D
:1009000083123408652399008316981C842C831263
:100910003308652399008316981C8B2C83123208A8
:10092000652399008316981C922C2030831299001D
:1009300008008301B0000730B0053008F000031054
:10094000F00D0310F00D0310700D813E9F00B101FA
:10095000B10A14303102031CA82CB301B401B20156
:100960001F151F19B12C1E08F300F20183161E0873
:10097000F000F1017208F0070318F10A7308F1079B
:1009800070088312B3070318B40A7108B407B20AD7
:1009900008303202031CB02C3408F1003308F00098
:1009A0000030F0070318F10AF030F107AF27CD301F
:1009B000F300CC30F4004330F50000277008B50098
:1009C0007108B6007208B7003508F0003608F1006B
:1009D0003708F200080083013008F3003108F40002
:1009E0003208F500F001C830F1004230F20038273B
:1009F00079277008B0007108B100B11F0B2D831664
:100A0000981CFF2C2D3083129900B009B109B00A4F
:100A10000319B10A112D8316981C0B2D2B3083124C
:100A200099003008B0003108B1003230B200D4254E
:100A30008316981C182D8312360865239900831697
:100A4000981C1F2D83123508652399008316981C66
:100A5000262D83123408652399008316981C2D2DAA
:100A60002E30831299008316981C332D831233087D
:100A7000652399008316981C3A2D8312320865234A
:100A800099008316981C412D20308312990008008C
:100A900083160313850103308600870183128501C5
:100AA0008601870151235B238023FF309200C530EC
:100AB000831692008C140B170B1601138312AA01D4
:100AC000AB019010101483160C148B170030831296
:100AD000B001B101B201A10803196B2DA1012B08CE
:100AE000F1002A08F000AF27C830F300CD30F40041
:100AF0003B30F50038277008B3007108B400720865
:100B0000B5002D08803AF000CE3070022130031974
:100B10002C02031C9E2D2308F1002208F00024085B
:100B2000F002031CF1032508F102AF27C530F300E2
:100B30002030F4003F30F5003827B02D2D08F100AB
:100B40002C08F000AF277008F3007108F400720859
:100B5000F5007030F0007530F1004730F2000027EA
:100B60007008B6007108B7007208B8003308B90001
:100B70003408BA003508BB000624F3012030F40025
:100B80004130F5003608F0003708F1003808F2006F
:100B900000277008B9007108BA007208BB00BD23B5
:100BA0006B2D8301800079281030F2002730F3008C
:100BB000831203133108F1003008F000B8277408DD
:100BC000B400B500B6011030F2002730F30036084B
:100BD000F1003508F00092237408B002031CB10341
:100BE0007508B102E830F2000330F3003108F1007B
:100BF0003008F000B8277408B300B500B601E8303B
:100C0000F2000330F3003608F1003508F0009223BB
:100C10007408B002031CB1037508B1026430F2001D
:100C2000F3013108F1003008F000B8277408B20071
:100C3000B500B6016430F200F3013608F100350862
:100C4000F00092237408B002031CB1037508B102CE
:100C50000A30F200F3013108F1003008F000B82743
:100C60007408B100B500B6010A30F200F30136088D
:100C7000F1003508F00092237408B002031CB103A0
:100C80007508B1023008B0003208043E84008313B6
:100C9000340880003208033E8400330880003208A4
:100CA000023E840032088000320A8400310880004D
:100CB00032088400300880000800840803190034DA
:100CC000720880008403710880008403700880002B
:100CD0000034F801710D720DF60076080319742EB8
:100CE000F80DF201F1170800F001F101F2010034F2
:100CF000F810740D750DF70077080319842E03188A
:100D0000F814F501F4170800F701F301F401F501F7
:100D1000080076080319742EF113F80C760CF20013
:100D20000318F1175D2EF608031DA72EF001F1013F
:100D3000F2015D2E72030319F00A0319F10A031977
:100D4000F20A0310F20CF10CF00CF60A932EF208E2
:100D5000031D9A2E700871040319962EF11B892E1B
:100D6000F6030319962E0310F00DF10DAE2E760842
:100D70007702031CC62E031908000310F20CF10CB5
:100D8000F00CF60A76087702BB2E0310F50CF40C73
:100D9000F30CF70A7608770603190800C52E803091
:100DA000F506840169267826B726781CDF2EF0091F
:100DB000F109F209F00A0319F10A0319F20AF81C01
:100DC000E92EF309F409F509F30A0319F40A0319E2
:100DD000F50A7308F00774080318740FF107750813
:100DE0000318750FF207F801F21F932EF009F109AD
:100DF000F209F00A0319F10A0319F20A7814932E82
:100E0000840169267826F901FA01FB01F608031925
:100E100008007708031908007602773EF600780C80
:100E2000F8061830F5000310F90DFA0DFB0D7208E5
:100E3000031D222F74087102031D202F73087002F6
:100E4000031C2C2F7308F0027408031C740FF102AA
:100E5000031CF20379140310F00DF10DF20DF50BE4
:100E6000132F7908F0007A08F1007B08F200932E26
:100E7000840169267826F901FA01FB010730F500A3
:100E80000310F40CF30C031C502F7008F9077108C1
:100E90000318710FFA0772080318720FFB0703108B
:100EA000F00DF10DF20DF50B402F0930F5005C2F20
:100EB0000310FB0CFA0CF90C0310F40CF30C031CDC
:100EC0006B2F7008F90771080318710FFA07720881
:100ED0000318720FFB07F50B582F7A307707F607C8
:100EE000780CF8067908F0007A08F1007B08F20027
:100EF000932E84016926F3018230F607F61B742EC7
:100F0000F030F607F61B952F183076020318742E72
:100F1000F608031D8E2F7818F2270800F603031039
:100F2000F00DF10DF20DF30D882F0310F20CF10C02
:100F3000F00CF60F952F8B2FF31FA12F7814F227AB
:100F4000A22FF8018E30F6008401F3080319932EC6
:100F50000310F30CF20CF10CF00CF60AA52FF201C1
:100F6000F11BF2037208F3009C2FF201F301A12F91
:100F7000F601F401F50172087304031DC22FF0019C
:100F8000F10100341F30F6040310F60AF20DF30DE0
:100F9000031CC52FF30CF20C73087102031DD22F32
:100FA00072087002031CDA2F7208F0027308031C27
:100FB000730AF102F40DF50DF60BF61ACA2FF61F9F
:100FC000E62FF409F40A0319F503F5097408F20091
:100FD0007508F300761F0034F009F00A0319F103D5
:100FE000F10900340310FF30F007F009031CF1078A
:100FF000F109031CF207F209031CF307F3090800C7
:00000001FF
